:100000000C9493010C94CB010C94CB010C94CB0178
:100010000C94CB010C94CB010C94CB010C94CB0130
:100020000C94CB010C94CB010C94101D0C94E21D8C
:100030000C9404180C94CB010C94CB010C94CB01C0
:100040000C94CB010C94CB010C94CB010C94CB0100
:100050000C94CB010C948C180C94CB010C94CB0118
:100060000C94CB010C94CB010C94CB010C94CB01E0
:100070000C94CB010C94CB010C94CB010C94CB01D0
:100080000C94CB010C94CB010C94CB010C94CB01C0
:100090000C94CB010C94CB010C94CB010C94CB01B0
:1000A0000C94CB010C94CB010C94CB017B047B040E
:1000B000A704A7040F052D05450645063805D105FB
:1000C000E205E2054F1E761E6E1F761E6E1FC21ED3
:1000D000E51E6E1F3C1F4B1F29001E001F00200045
:1000E00021002200230024002500260027002D00E7
:1000F0002E002A002B0014001A000800150017001B
:100100001C0018000C00120013002F0030003100FA
:10011000390004001600070009000A000B000D005A
:100120000E000F003300340028004C00E1003100C5
:100130001D001B000600190005001100100036000C
:1001400037003800E5000151E000E300E200000064
:10015000000000002C00000000000000E600E700A6
:100160006500E400005C01000100010001000100E5
:100170000100010001000100010001000100010077
:100180000100010001000100010001000100010067
:100190000100010001000100010001000100010057
:1001A0000100010001000100010001000100010047
:1001B0000100010001000100010001000100010037
:1001C0000100010001000100010001000100010027
:1001D000010001000100010001000000000000001A
:1001E000010000000000000001000100010001000A
:1001F0001203490072006900730052006500760026
:1002000030000000140353006F006E004F006600C2
:100210004100720065007300000004030904090234
:100220003B00020100A0FA090400000103010100E3
:100230000921110100012240000705810308000186
:10024000090401000103000000092111010001223D
:100250007B0007058203200001120100020000005C
:10026000084B49313001000102000105010902A1DA
:100270000185020901A100050919012908150025B8
:1002800001950875018102050109300931158125A3
:100290007F95027508810609381581257F950175BE
:1002A000088106050C0A38021581257F950175081D
:1002B0008106C0C005010980A101850319012AB783
:1002C00000150126B700950175108100C0050C09C5
:1002D00001A101850419012AA002150126A0029599
:1002E0000175108100C005010906A101050719E08B
:1002F00029E715002501950875018102950175080A
:1003000081010507190029FF150026FF00950675D4
:1003100008810005081901290595057501910295C7
:100320000175039101C011241FBECFEFDAE0DEBFDB
:10033000CDBF04B603FE18C080917602909177027B
:10034000A0917802B09179028730904BA740B04BD2
:1003500059F410927602109277021092780210925D
:100360007902E0E0F8E3099511E0A0E0B1E0E2E411
:10037000F0E402C005900D92AE38B107D9F722E043
:10038000AEE8B1E001C01D92A637B207E1F70E94C6
:100390004D120C941F200C94000081E0089581E020
:1003A00008950C94CF0108950C94D3011F93CF931B
:1003B000DF9300D000D01F92CDB7DEB749835A83B8
:1003C0006B833091910189819A81311114C0662328
:1003D00059F0222349F00E948208182F682F898142
:1003E0009A810E942B0803C00E945608182F698129
:1003F0007A81812F04C00E94820869817A810F90DE
:100400000F900F900F900F90DF91CF911F910C9450
:10041000B80FFC01262F4081518162817381848154
:100420000C94D60181E00895CF93DF93EC0160E056
:100430000E940902BE01DF91CF910C94D4010C946B
:10044000FE100C94FA1008950E94D5060E94230213
:100450002FEF84E39CE0215080409040E1F700C002
:1004600000000C94B2180F931F93CF93DF938C016D
:1004700061E00E940902EC01B8010E94D1018823C9
:10048000F1F1B801CE010E94CF168823C1F1B80165
:10049000CE010E94E314882391F1B801CE010E949D
:1004A0002B16882361F1F8018281882309F1CB356D
:1004B0008DE5D807C1F050F4C115FCE5DF0781F0E8
:1004C000CF3DDC45A9F40E94B90D19C0CC35EDE54E
:1004D000DE0761F0CD35DD4559F40E94FC0C08C003
:1004E0000E9424020CC00E94050D02C00E94080D4B
:1004F000C801DF91CF911F910F910C94CD0180E045
:10050000DF91CF911F910F9108950E94E6170C94EF
:100510009E020E94A1020C94EC1708950C948D0287
:1005200081E008950C9490020895CF93C82F0E9403
:100530008E028C2F0E949202CF91089580E00C943D
:1005400095020E942B170C9495020E942B179091F4
:100550009001891721F0809390010C9495020895E1
:10056000CF93DF93CDB7DEB72B970FB6F894DEBFEE
:100570000FBECDBF4F83588769877A878B876111FC
:100580000E94480C9E012F5F3F4F86E0F9011192B7
:100590008A95E9F785E0FE013796D90101900D9221
:1005A0008A95E1F789819A814C815D81452B31F0F3
:1005B0009F3F31F491E08F3F19F403C091E001C0F7
:1005C00090E090FF09C049815A816B817C818D81C7
:1005D0009E810E94690B05C0C9010E94120281110F
:1005E000F2CF2B960FB6F894DEBF0FBECDBFDF91D2
:1005F000CF910895FC01808191810E94C4080895E3
:10060000CF93882309F4A4C0C82F8238C1F40E9474
:100610002B1781FD9DC069E3809102019091030138
:100620000E94BE170E946A0C2FEF81EE94E02150C9
:1006300080409040E1F700C0000069E319C08338B2
:1006400001F50E942B1780FD83C063E580910201B4
:10065000909103010E94BE170E946A0C2FEF81EE59
:1006600094E0215080409040E1F700C0000063E535
:1006700080910201909103010E94C017CF910C94C8
:100680006A0C8438C1F40E942B1782FD61C067E4B4
:1006900080910201909103010E94BE170E946A0C92
:1006A0002FEF81EE94E0215080409040E1F700C0B0
:1006B000000067E4DDCF8CEF8C0F813AD0F46C2F13
:1006C00080910201909103010E948817882349F0CC
:1006D0006C2F80910201909103010E94C0170E942B
:1006E0006A0C6C2F80910201909103010E94BE1749
:1006F000C5CF80E28C0F883048F4C77081E001C01C
:10070000880FCA95EAF70E942B0CB8CFEBE5EC0FE7
:10071000E33040F4F0E0E95BFE4F808190E0CF9160
:100720000C945017E8E5EC0FE73150F4F0E0EE0FD1
:10073000FF1FE75EFE4F80819181CF910C94661779
:10074000CD3E30F08C2F0E94D212CF910C94A41386
:10075000CF910895882309F464C0823879F40E9407
:100760002B1781FF5EC069E3809102019091030124
:100770000E94BE170E946A0C69E310C08338B1F46E
:100780000E942B1780FF4DC063E58091020190917C
:1007900003010E94BE170E946A0C63E5809102016A
:1007A000909103010E94C0170C946A0C843879F46C
:1007B0000E942B1782FF35C067E48091020190915F
:1007C00003010E94BE170E946A0C67E4E7CF9CEF0A
:1007D000980F913A10F4682FE1CF90E2980F98307B
:1007E00050F4877091E001C0990F8A95EAF7892F3C
:1007F0000E94310CD9CF9BE5980F933020F480E014
:1008000090E00C94501798E5980F973120F480E011
:1008100090E00C9466178D3E20F00E942D130C94EE
:10082000A41308951F93CF93DF93182FEB010E9419
:100830000003209741F08FE99FE00197F1F700C096
:1008400000002197F6CF812FDF91CF911F910C945B
:10085000AA03893319F060E070E002C060E570E03F
:100860000C941204882321F00E942B0C0C946A0C27
:100870000895882321F00E94310C0C946A0C08958D
:10088000CF92DF92EF92FF920F931F93CF93DF935C
:100890007C01D62FC72FFC011281058102950F70B4
:1008A0000E94210C8823B9F01123A9F08C2F807F9E
:1008B000803421F080E28D0F883068F08091500202
:1008C00082FD09C082E00E94CA0C0E94210C91E0C6
:1008D000D82ED92601C0D12CCC2EC2948FE0C822AC
:1008E0008C2D90E08C30910508F0CFC1FC01EA5AC4
:1008F000FF4F0C94B61F8C2F807FCF70882311F090
:10090000C295C07F112399F0CC2309F4AAC180E2DB
:100910008D0F883010F0D11104C08C2F0E942B0C49
:1009200003C08C2F0E943B0C0E946A0C9AC18D2F31
:100930000E94AA03CC2309F4A8C180E28D0F88305D
:1009400038F1DD2329F18C2F0E94410C24C08C2F1B
:10095000807FCF70803211F0C295C07FDD2319F007
:10096000D130A1F13DC08091500282FF17C0112308
:1009700049F0CC2329F08C2F0E942B0C0E946A0C8A
:1009800080E070C180E00E94AA03CC2309F47DC1FD
:100990008C2F0E94310C0E946A0C77C1112371F0D8
:1009A000002341F0013031F40E944B0C8C2B0E944B
:1009B000530C6BC10E944B0C8C2B1DC0002319F0F3
:1009C000013009F462C10E94600C25C0112321F09E
:1009D000063008F05AC10EC0053008F056C11BC0E1
:1009E000112361F0002331F0F701858180FF39C1C7
:1009F0008F7085838C2F0E94320447C1002359F0E9
:100A0000D93309F03FC1FFEF07EE13E0F15000408A
:100A10001040E1F735C18C2F0E94390436C18C2F6C
:100A200086958695837019F0813061F02EC111236F
:100A300021F08D2F9C2F937002C080E090E00E94E7
:100A400050172BC1112321F08D2F9C2F937002C0C2
:100A500080E090E00E94661720C18D2F112319F0CD
:100A60000E94D21202C00E942D130E94A41315C12D
:100A70008C2F837009F047C011110BC12D2F2295C7
:100A800026952770220F220F6D2F6F70862F90E012
:100A9000A0E0B0E0022E04C0880F991FAA1FBB1F60
:100AA0000A94D2F7D4FF10C04FE050E060E070E04D
:100AB00004C0440F551F661F771F2A95D2F7409533
:100AC00050956095709503C040E050E0BA01C6951E
:100AD000C695C3708A019B01082B192B2A2B3B2B2F
:100AE000C901B801C23049F058F4C13019F00E9470
:100AF0004107CFC00E942F07CCC00E945307C9C036
:100B00000E942D07C6C0112319F08C2F817001C0DF
:100B10008695882309F4BDC02D2F22952695277030
:100B2000220F220F6D2F6F70862F90E0A0E0B0E0B3
:100B3000022E04C0880F991FAA1FBB1F0A94D2F768
:100B4000D4FF10C04FE050E060E070E004C0440FFC
:100B5000551F661F771F2A95D2F7409550956095CF
:100B6000709503C040E050E0BA01C695C695C370C9
:100B70008A019B01082B192B2A2B3B2BC901B80199
:100B8000C23049F058F4C13019F00E94060881C003
:100B90000E94F4077EC00E9418087BC00E9467076D
:100BA00078C0CF70112339F08C2F0E948D078D2FC4
:100BB0000E9432046EC08D2F0E9439048C2F0E9437
:100BC000AE0767C0D23F21F128F4D03F41F0D13FBA
:100BD000C1F043C0D33F19F1D43F79F03EC0112397
:100BE00041F0053008F051C08C2F8F710E94D3075F
:100BF0004CC0063008F049C0F7CF8091500282FF08
:100C000018C0112339F08C2F8F710E948D073DC0C1
:100C10001123C9F38C2F8F710E94AE0736C01123A8
:100C200029F08C2F8F710E9478072FC00E947307C4
:100C30002CC0112349F0CF718C2F0E948D0763E0E7
:100C40008C2F0E94AF0C21C081E00E94CA0C0230A0
:100C5000E0F082E00E94CA0C18C0112331F000239A
:100C600091F28D2F0E94000310C0002399F2D93316
:100C700049F41FEF27EE33E0115020403040E1F7F8
:100C800000C000008D2F0E94AA0388EF8C0D8430D5
:100C900020F40E942B170E949502DD20C9F00E94CB
:100CA0001D0C80FD15C0F70112820E94170C0E94D6
:100CB0008D07C7010E9489060E94170CDF91CF9112
:100CC0001F910F91FF90EF90DF90CF900C94AE07A3
:100CD000DF91CF911F910F91FF90EF90DF90CF9018
:100CE00008950F931F93CF93DF93EC01688179816F
:100CF0008A810E94CF088C010E942A080E941B074B
:100D0000B801CE010E944004DF91CF911F910F9155
:100D10000895CF93DF93EC01988189812B813C81E9
:100D2000232B31F08F3F31F481E09F3F19F403C052
:100D300081E001C080E080FD1DC0CE010E94330231
:100D4000811110C00E94210C8823A1F08A81882380
:100D500089F08091500282FD0DC082E0DF91CF9139
:100D60000C94CA0CCE010E947106CE01DF91CF9186
:100D70000C941402DF91CF91089580E090E00E94DE
:100D8000501780E090E00E9466170E94480C0E9475
:100D90006A0C0E94D5140C94A413809102019091C6
:100DA00003010E94C2170C94BD060E94380C0C94DB
:100DB000CD0692959F70963079F010F4925001C054
:100DC0009A50923068F4803F69F018F4883E40F4FD
:100DD00009C0843F29F406C0883E20F0813F11F00D
:100DE00080E0089581E00895FC01808191810E9456
:100DF000C4080E94D9060895CF93DF9300D000D095
:100E00001F92CDB7DEB70F900F900F900F900F90FD
:100E1000DF91CF910895CF93DF9300D000D000D021
:100E2000CDB7DEB726960FB6F894DEBF0FBECDBFA6
:100E3000DF91CF910895089508950C941C070C94A8
:100E40001D070E941F076093C3017093C401809324
:100E5000C5019093C6010C94BD060C9421070F9315
:100E60001F930091C3011091C4012091C5013091DD
:100E7000C601602B712B822B932B1F910F910C9429
:100E800021070F931F930091C3011091C40120917A
:100E9000C5013091C60160237123822393231F91E2
:100EA0000F910C9421070F931F930091C301109190
:100EB000C4012091C5013091C601602771278227A6
:100EC00093271F910F910C9421070C941C070E94EB
:100ED00065076093BF017093C0018093C101909337
:100EE000C2010C94BD0660E070E0CB010C94670772
:100EF0000F931F9341E050E060E070E08A019B0196
:100F000004C0000F111F221F331F8A95D2F7C90199
:100F1000B8011F910F910C9467070F931F9341E045
:100F200050E060E070E004C0440F551F661F771F5B
:100F30008A95D2F78091BF019091C001A091C10123
:100F4000B091C2018A019B01082B192B2A2B3B2B44
:100F5000C901B8011F910F910C9467070F931F935C
:100F600041E050E060E070E004C0440F551F661F90
:100F7000771F8A95D2F7409550956095709580912E
:100F8000BF019091C001A091C101B091C2018A013D
:100F90009B01082319232A233B23C901B8011F9170
:100FA0000F910C9467070F931F9341E050E060E0AE
:100FB00070E004C0440F551F661F771F8A95D2F753
:100FC0008091BF019091C001A091C101B091C20177
:100FD0008A019B01082719272A273B27C901B80145
:100FE0001F910F910C9467070F931F930091BF01FE
:100FF0001091C0012091C1013091C201602B712B71
:10100000822B932B1F910F910C9467070F931F93C3
:101010000091BF011091C0012091C1013091C20126
:1010200060237123822393231F910F910C946707F0
:101030000F931F930091BF011091C0012091C10136
:101040003091C20160277127822793271F910F914A
:101050000C94670708952EE0929F800D1124E82FCD
:10106000E695E695E695877051E001C0550F8A95A3
:10107000EAF785E0E89FF0011124EE56FE4F20E0EC
:1010800030E070E04081CB01022E02C0969587953A
:101090000A94E2F7817081958427852384278193C0
:1010A0002F5F3F4F2530310569F708952EE0929F5D
:1010B000800D1124682F669566956695982F977018
:1010C00085E0689FB001112440E050E080E0FB0122
:1010D000E40FF51FEE56FE4F208130E0092E02C0CE
:1010E000369527950A94E2F721703327042E01C024
:1010F000220F0A94EAF7822B4F5F5F4F453051056C
:1011000031F70895BF92CF92DF92EF92FF920F9343
:101110001F93CF93DF938C01C090BF01D090C0018B
:10112000E090C101F090C2018091C3019091C4018F
:10113000A091C501B091C601C82AD92AEA2AFB2A82
:10114000CFE1D0E0D701C6010C2E04C0B695A7951B
:10115000979587950A94D2F780FD04C0219790F760
:10116000B12C07C0BC2EB8018C2F0E94CB0F019769
:10117000A9F38B2DDF91CF911F910F91FF90EF90ED
:10118000DF90CF90BF900895CF93DF93EC010E9442
:101190008208BE010E94CB0FDF91CF9108951F936B
:1011A000CF93DF93EB0190919101992321F0CB0133
:1011B0000E94C40813C0882349F0CB010E94820812
:1011C000182F682FCE010E942B0804C0CB010E946B
:1011D0005608182FBE01812F0E94CB0FDF91CF91AF
:1011E0001F9108951F93CF93DF93C091C70116E01D
:1011F0008091C801C81799F0D0E01C9FF0011D9F95
:10120000F00D1124E753FE4F4081518162817381BB
:10121000848195810E940B072196C770E9CFDF91E9
:10122000CF911F9108954091F9015091FA01609179
:10123000FB017091FC018091FD019091FE010C94E5
:101240000B07EF92FF920F931F93CF93DF93809141
:10125000FE0182958F7009F065C08091FB018823A3
:1012600009F460C08091C701F090C8011091F901A4
:101270000091FA016091FC017091FD0191E01F3F26
:1012800009F090E0C0910001D0910101292F96E072
:10129000E92E8F1509F446C06115710521F00F3F45
:1012A00021F030E003C031E001C0322F90E030FD8A
:1012B00036C0E89EF001E99EF00D1124DF01A7532E
:1012C000BE4F11963C911197301329C03C913113B8
:1012D00026C012963C911297311121C013964D9160
:1012E0005C911497461B570B4C175D07C0F4809117
:1012F000FE018F7080618093FE01E253FE4F80817A
:101300008F708061808389EF91E00E948906DF9170
:10131000CF911F910F91FF90EF900C94F2080196DE
:101320008770B7CFDF91CF911F910F91FF90EF9012
:1013300008959F92AF92BF92CF92DF92EF92FF9269
:101340000F931F93CF93DF93CDB7DEB761970FB69F
:10135000F894DEBF0FBECDBF8C0185E0F801DE0141
:101360001D9601900D928A95E1F7D8011296EC90A6
:101370009091F901E091FA012091FC013091FD0179
:101380002115310531F0EF3F31F481E09F3F19F431
:1013900003C081E001C080E0B82FB1709B2E80FDBA
:1013A00047C1D8014C9111965C9111971396AD905D
:1013B000BC90149789EFC82E81E0D82EF090FB01E5
:1013C000B501621B730B2091000130910101FF20D8
:1013D00009F4D9C08091FE016217730708F095C027
:1013E000282F207F09F052C05E1313C0491311C08B
:1013F000FE2CE1100EC08F7080618093FE010E9470
:101400001309C6010E9489068091FE01F8018583B7
:101410004DC1AB2831F05F3F31F481E04F3F19F40B
:1014200003C081E001C080E080FD03C081E08E2523
:1014300002C080E090E0F82FF170FF2E80FF1CC00A
:101440008091C7012091C80136E0821709F40BC1D1
:1014500090E0389FF001399FF00D1124E753FE4FC3
:101460006181561306C06081461303C06281E61293
:1014700003C001968770E9CFFE2CEE2009F416C157
:101480008091FE0181608093FE0154C05E1306C00E
:10149000491304C0E11002C0F80199C0C8010E94BC
:1014A000F406882361F1EE2051F12091FE01822F94
:1014B00082958F7090E0029774F08091F90190917D
:1014C000FA0198878F831986BB86AA862C87CE015E
:1014D00007960E94890686E0F801A9EFB1E0019025
:1014E0000D928A95E1F70E9421090E9413090AC012
:1014F0005E1711F1C8010E94F40681112CC0C801C9
:101500000E948906FF24F394D1C0282F207F81F701
:101510007A2DB98AA88A6E2D89890E94FC0689EFE6
:1015200091E00E94890686E0D6011D928A95E9F72E
:101530000E941309F12CBAC04913DCCFE110DACFB5
:10154000F8018583C8010E94890686E0D6011D92B4
:101550008A95E9F7ABC0EE2091F22091FE01822F2F
:1015600082958F7090E002970CF4B5CF8091F901CD
:101570009091FA019A8389831B82BD82AC822E836B
:10158000CE010196A6CF6217730708F044C0FE2C67
:10159000EE2009F4B4CF5E1330C049132EC0209161
:1015A000FE0120FD21C0822F82958F70482F50E0D0
:1015B00041155105C9F0F80125834F30510541F01F
:1015C0008F5F982F9295907F822F8F70892B8583C4
:1015D000C8010E94890686E0F801A9EFB1E00190F8
:1015E0000D928A95E1F73CC086E0F801A9EFB1E0E1
:1015F00001900D928A95E1F759C0C8010E94F40646
:10160000811169CF8091FE0181608093FE01C80144
:101610000E9489064BC07A2DB98AA88A6E2D8989C5
:101620000E94FC0686E0D6011D928A95E9F718C053
:10163000EE2009F464CFC8010E94F406F82E882336
:1016400009F45DCF86E0F801A9EFB1E001900D92B9
:101650008A95E1F789EF91E00E94FA020E94210940
:101660000E94130923C04D875E878D859E850E9449
:10167000C408292F22952F70223028F49F7039F04A
:10168000811105C00BC0243028F49F7049F4805E9E
:10169000883020F0C8010E9489069F2CF92C06C0D2
:1016A000D80115969C91907F91F7F8CF8F2D619678
:1016B0000FB6F894DEBF0FBECDBFDF91CF911F9163
:1016C0000F91FF90EF90DF90CF90BF90AF909F90E1
:1016D00008951F93CF93DF93CDB7DEB72C970FB646
:1016E000F894DEBF0FBECDBF4F83588769877A87D6
:1016F0008B879C87CE0107960E9499098823D1F099
:101700009F8188852A853B85232B31F08F3F31F4DB
:1017100081E09F3F19F403C081E001C080E080FDBB
:1017200047C04F81588569857A858B859C850E9445
:101730000B073EC086E0FE013796DE011196019050
:101740000D928A95E1F7FF81E8856A857B856115B1
:10175000710531F0EF3F31F481E0FF3F19F403C030
:1017600081E001C080E080FD23C02091C80130E00D
:10177000C9010196877099274091C70150E08417ED
:101780009507F1F1F983EA837D836C8396E0929F5C
:10179000D001939FB00D1124A753BE4FFE01319687
:1017A00001900D929A95E1F78093C8010E94F2088A
:1017B00016E08091C7019091C801891771F1189FB7
:1017C000C001112487539E4F0E949909882329F153
:1017D000E091C7011E9FF0011124E753FE4F4081A5
:1017E000518162817381848195810E940B07809170
:1017F000C70190E00196877099278093C701D9CFE0
:101800000E94D5061092C8011092C701E9EFF1E0DD
:1018100086E0DF011D928A95E9F72C960FB6F894C1
:10182000DEBF0FBECDBFDF91CF911F910895809194
:1018300007028595859585950895809107028770A3
:10184000089590910702977081E009F480E008956F
:1018500080911202089590911202892B80931202B6
:101860000895809590911202892380931202089521
:1018700010921202089590911102892B8093110207
:101880000895809590911102892380931102089503
:1018900010921102089580910802089508950C9401
:1018A0004E0C0C944F0C9091500292FD08C09091F8
:1018B0000802981721F0809308020C94510C0895A7
:1018C00080910802882329F01092080280E00C948D
:1018D000510C0895CF93DF93E0910201F091030141
:1018E000809112028083E0910201F09103019081C6
:1018F00080911102892B808380910802882381F0D6
:10190000E0910201F09103019081892B8083809105
:101910000201909103010E947C1781110E94600CCA
:10192000C0910201D091030148E050E06FEF71E0F7
:10193000CE010E94D01F892B69F088E0FE01AFEF35
:10194000B1E001900D928A95E1F7CE01DF91CF9140
:101950000C943717DF91CF9108950C944E0C909111
:10196000500292FD10C098E0899F90011124262B0F
:10197000209307020E948D07809107028595859527
:1019800085950C94AD0C0C948D071092070280E0A5
:101990000C94AD0C2091070280958223809307025E
:1019A000982F977099F430E0482F082E000C550BB3
:1019B0002417350759F09091500292FD07C0859584
:1019C000859585950E94AE070C94C50C089590915D
:1019D000500292FB222720F9281769F080FB92F928
:1019E0009093500280914F02909150020E94350DC9
:1019F00082E00C94CA0C08958091500282FB8827E3
:101A000080F991E089270C94E70C81E00C94E70CB5
:101A100080E00C94E70C6FEF7FEF80E090E00C9497
:101A2000092080E090E00E94E51F21E0893E9E4F62
:101A300009F020E0822F089582E090E00C94DD1FF1
:101A400083E090E00C94DD1FCF9384E090E00E944F
:101A5000DD1FC82F82E290E00E94DD1F2C2F30E0B6
:101A6000A901582BCA01CF910895CF93C92F682F90
:101A700084E090E00E94EB1F6C2F82E290E0CF9117
:101A80000C94EB1FAB01BC018FE090E00C94FD1FA8
:101A9000AB01BC0183E190E00C94FD1F60E070E0BD
:101AA000CB010C94480D60E070E0CB010E94420D28
:101AB0000C944E0D69EE7EEF80E090E00E940920CC
:101AC00060E082E090E00E94EB1F60E083E090E045
:101AD0000E94EB1F1092C3011092C4011092C50125
:101AE0001092C60160E084E090E00E94EB1F60E08D
:101AF00082E290E00E94EB1F60E085E090E00E94AF
:101B0000EB1F60E086E090E00E94EB1F6FEF87E044
:101B100090E00E94EB1F40E050E0BA0188E090E0C6
:101B20000E94FD1F60E08DE090E00E94EB1F40E00E
:101B300050E0BA0188E190E00E94FD1F60E087E17B
:101B400090E00E94EB1F40E050E0BA018CE190E091
:101B50000E94FD1F60E070E080E290E00E9409209A
:101B600040E050E0BA0188E190E00E94FD1F0C9433
:101B7000530D0C945A0D682F8EE090E00C94EB1FDF
:101B80000E947118609321027093220280932302B5
:101B90009093240260931D0270931E0280931F0293
:101BA00090932002089585B7806885BF85B78068C7
:101BB00085BF089581E008950C94DA0D08950C9482
:101BC000DE0D0C94DE0D0C94E10D0C94DE0D0C94E6
:101BD000E50D0C94DE0D0E94D30D87EA90E10E9482
:101BE00021170E94E90D0C94E70D0E94DF0D0C9463
:101BF000DE0D0E94C1100C9494020E945C180E9499
:101C0000A6110E94F90D0C94E30D5F926F927F92E2
:101C10008F929F92AF92BF92CF92DF92EF92FF92FC
:101C20000F931F93CF93DF93CDB7DEB72A970FB6ED
:101C3000F894DEBF0FBECDBF0E94BB11C82E81112C
:101C40000E94C00D33E1832E32E0932E00E010E0BD
:101C5000502E802F0E94E5105C01F401619071907C
:101C60004F016826792661147104B1F40F5F1F4F8C
:101C70000530110569F78FEF89838A831B820E94E3
:101C800065188160782F9D838C8349815A816B818F
:101C90008D810E94B0023AC08091250281FD0E9490
:101CA000EE10D12CEE24E394F12CC3018E219F2160
:101CB000892B29F10E94DC0D8823A9F0DE825F8246
:101CC000AE20BF2081E0AB2809F480E088870E9425
:101CD00065188160782F9A8789874E815F81688532
:101CE0008A850E94B002000F111FF801ED5EFD4FC2
:101CF00080819181E826F926F182E08207C0D394A1
:101D0000EE0CFF1CFEE0DF12D0CFB0CF81E0C1109F
:101D100001C080E02A960FB6F894DEBF0FBECDBF9B
:101D2000DF91CF911F910F91FF90EF90DF90CF90B7
:101D3000BF90AF909F908F907F906F905F9008952D
:101D40000E94050E0E94C2130C94A502CF93DF934C
:101D50000E94D00FEC01811521E5920708F045C0E3
:101D6000811530E5930708F094C0883E910528F569
:101D7000803E910508F0F8C0883A910570F4853AE4
:101D8000910508F07CC08130910509F475C008F414
:101D9000E8C0049708F0E8C0E4C08F3B910508F064
:101DA000E0C0C85AD0E0CC0FDD1FC65BDE4F099003
:101DB000D881C02DCE019464D8C0811540E294072B
:101DC00058F4811551E0950708F0CEC08D3E91057D
:101DD00008F4C7C09065C9C0C11580E4D80708F4ED
:101DE000C0C0DF70CE01906AC0C0811525E59207A2
:101DF000A8F4811534E5930708F095C0811543E5F3
:101E0000940708F07BC0811552E5950708F061C082
:101E1000D82FCC27CE01816F906AA7C0C11589E564
:101E2000D807A0F4C11528E5D20708F082C0C11573
:101E300036E5D30708F095C08C2F0E9464108F718F
:101E400090E0D82FCC27CE0190628FC0C1154AE513
:101E5000D40708F474C0CE0190568115904208F062
:101E600080C08D2F8F710E946410DD27D0628F712A
:101E7000AE01582BCA0179C081E090E076C0C55A06
:101E8000D0E0C858DE4F8881C82FD0E0CE019064E2
:101E90006CC074E0969587957A95E1F7282F2370AA
:101EA0003C2F337081E090E002C0880F991F3A9573
:101EB000E2F79C68AC01522B9A019C2F9F7096957B
:101EC000969550E2959FE0011124C9018C2B9D2B22
:101ED0004CC08370992721E030E002C0220F331FED
:101EE0008A95E2F79C2F9695969580E2989FE0015F
:101EF0001124C22BD32BCE019C6837C08370992745
:101F000021E030E002C0220F331F8A95E2F79C2FB8
:101F10009695969540E2949FE0011124C22BD32B15
:101F2000CE019A6822C0D82FCC27CE01846F906A48
:101F30001CC0DC2FCC27CE01806F906A16C08C2F7E
:101F40008F700E94641094E0D695C7959A95E1F73A
:101F5000CF70D0E0DC2FCC27D0699E01282BC9019F
:101F600004C080E090E001C0CE01DF91CF910895E0
:101F700026E4829FC0011124FC012EE0729FE00D37
:101F8000F11D1124E60FF11DEE0FFF1FE852FF4F68
:101F90008591949108950E94B80F0E94A60E08950D
:101FA0008238910569F1B0F48133910509F46DC06F
:101FB00048F48932910509F463C08A32910509F425
:101FC00069C008958533910509F455C08933910599
:101FD000B9F00895833E910569F138F4803E91058A
:101FE000B1F0823E910509F10895863E9105A9F16F
:101FF000873E9105B9F1843E910509F064C023C084
:1020000020914F0220FD4FC021FD4DC008958091C9
:102010004F0280FD44C08091500280FF44C08091F7
:102020004F0284FD42C083EE4DC080914F0282FF7B
:1020300038C0F5CF80914F0282FD33C080915002AD
:1020400080FD31C0ECCF8091500281FF32C0809181
:102050004F0284FD2AC087EE35C080914F0283FF76
:1020600026C0F5CF80914F0283FD21C080915002A0
:1020700081FD1FC0ECCF80914F0285FD1CC01DC0AB
:1020800080914F0285FD19C016C080914F0286FDD8
:1020900016C017C080914F0286FD13C010C089E39F
:1020A00011C082EE0FC080EE0DC080E00BC086EE46
:1020B00009C084EE07C089E205C085E303C08AE257
:1020C00001C081E390E0089590914F0292FF0DC00E
:1020D000282F2871283019F4877F846006C0282FA4
:1020E0002471243011F48B7F886093FF0DC0282F5A
:1020F0002871283119F4877E846106C0282F247145
:10210000243111F48B7E88612091500220FF0DC094
:10211000382F3871383019F4877F816006C0382F26
:102120003171313011F48E7F886021FF0DC0282F6E
:102130002871283119F4877E816106C0282F21710A
:10214000213111F48E7E886194FD877E089580E0B0
:1021500008950C940B0D0E94BB118FE39CE901972D
:10216000F1F700C000000E94BB1180E00E94E51062
:1021700080FF04C00E94A9100C94B21808950C941A
:10218000AB100E94110D811102C00E94B90D0E9476
:102190001C0D809325020E94240D90935002809381
:1021A0004F020E94BF100E94200D682F70E080E057
:1021B00090E00E942D076091BF017091C001809155
:1021C000C1019091C2010C946507E82FF0E0EE0F79
:1021D000FF1FE55AFD4F808191810895089580EA9F
:1021E0008A95F1F7089500C008950C94EF100895B2
:1021F0000C94F7100C94F8100C94F7100C94FC103D
:10220000F894E82FE295EF70F0E031A1282F2F70BD
:1022100081E090E001C0880F2A95EAF7982F909509
:10222000932391A392A1892B82A3789408950F936D
:102230001F93CF93DF93C9E8D1E089918F3F11F0CD
:102240000E94001181E0CE38D807B9F7CBE7D1E082
:1022500009E811E089918F3F11F00E9400110C17DD
:102260001D07C1F7DF91CF911F910F910895BF9284
:10227000CF92DF92EF92FF920F931F93CF93DF9352
:102280008C01C62FD0E0CE0187579E4F6C01FC0118
:1022900090819F3F09F450C0B62EF894E92FE29543
:1022A000EF70F0E081A19F7021E030E001C0220FCB
:1022B0009A95EAF7822B81A382A12095282322A355
:1022C00078940E94F310EBE7F1E049E851E021E057
:1022D00030E0E12CF12C61916F3F89F0A62FA2959F
:1022E000AF70B0E090968C9190E06F7002C09595C1
:1022F00087956A95E2F780FD02C0C90102C080E0BF
:1023000090E0E82AF92A220F331F4E175F0719F7CA
:10231000F60180818F3F11F00E94001161E0E1140D
:10232000F10409F460E08B2D0E94F510CC0FDD1F45
:10233000C00FD11FF982E882DF91CF911F910F91D9
:10234000FF90EF90DF90CF90BF9008950E941711FB
:102350008AE0EBE5F2E0DF01982F1D929A95E9F70C
:10236000E1E5F2E0DF011D928A95E9F785E00E9440
:1023700006120C941F02FF920F931F93CF93DF93CB
:10238000CDB7DEB72A970FB6F894DEBF0FBECDBF2C
:102390008E010F5F1F4F8AE0F80111928A95E9F7CD
:1023A000F12C6F2DC8010E943711F394F5E0FF1254
:1023B000F8CF4AE050E0B80181E592E00E94D01FDA
:1023C000FF24F394009709F4F12C892B41F08AE063
:1023D000F801A1E5B2E001900D928A95E1F72F2D69
:1023E00045E06BE572E081E592E00E9407120E94F1
:1023F00021028F2D2A960FB6F894DEBF0FBECDBFF7
:10240000DF91CF911F910F91FF9008950895FF9252
:102410000F931F93CF93DF93F82E092F162FD72FEB
:10242000C42F222349F081E0809328020E9465187E
:102430009093270280932602809128028823D9F066
:1024400080912602909127020E947D18059798F0AE
:10245000EF2DF02FA12FBD2F80E090E04C2F50E00A
:102460008417950734F4219131912D933D93019672
:10247000F7CF10922802DF91CF911F910F91FF901B
:1024800008950E94681A0E94FD0D0C94741A0E940F
:10249000781A0E94A00E0C94921A0E9403180E94AF
:1024A0004F1A0E94EB0D0E9441120E9447120E9497
:1024B000F50DFBCF80912F0280FF06C060910901CE
:1024C00070E0660F771F26C081FF04C0609109018C
:1024D00084E005C082FF07C06091090188E0689F21
:1024E000B001112417C090912E029923D1F0609170
:1024F0000801961788F72091090188E0289F90012C
:102500001124929FA001939F500D112470E0CA01E5
:102510000E94A21F6038710540F46115710519F41D
:1025200006C068E070E0862F08958FE7089581E087
:10253000089580912F0280FF08C06091050170E02E
:10254000759567957595679521C081FF06C0609167
:10255000050170E07595679519C082FF04C0609110
:10256000050170E010C090912D02992399F06091BF
:1025700004019617A0F780910501899FC0011124DD
:1025800070E00E94A21F6038710540F4611571056A
:1025900019F406C061E070E0862F08958FE7089572
:1025A00081E008958D3E21F40E945A12819504C065
:1025B0008E3E29F40E945A128093330208958F3E72
:1025C00021F40E945A12819504C0803F29F40E9490
:1025D0005A12809332020895893F19F40E94991289
:1025E00005C08A3F31F40E9499128195809334028C
:1025F00008958B3F21F40E949912819504C08C3F6D
:1026000029F40E9499128093350208959FE0980F53
:10261000983078F421E030E0A90102C0440F551F42
:102620009A95E2F7CA0190913102892B8093310289
:1026300008958D3F21F480912F0281600BC08E3F61
:1026400021F480912F02826005C08F3F29F4809190
:102650002F02846080932F0208958D3E39F490916B
:10266000330297FF35C01092330259C08E3E29F4D1
:10267000909133021916BCF32BC0909132028F3E19
:1026800029F497FF25C01092320249C0803F19F407
:102690001916CCF31DC090913402893F29F4191604
:1026A000BCF4109234023BC08A3F19F497FF10C06B
:1026B000F8CF8B3F39F49091350297FF09C0109203
:1026C00035022DC08C3F21F4909135021916BCF3D0
:1026D0009FE0980F983080F421E030E0A90102C01B
:1026E000440F551F9A95E2F7CA01809590913102E7
:1026F00089238093310213C08D3F21F480912F02F2
:102700008E7F0BC08E3F21F480912F028D7F05C0FC
:102710008F3F29F480912F028B7F80932F0280912D
:102720003202811106C080913302811102C01092E1
:102730002E0280913402811106C0809135028111F0
:1027400002C010922D0208950E9465182091320255
:10275000211104C020913302222321F090932C02F6
:1027600080932B0220913402211104C02091350264
:10277000222321F090932A028093290280E392E0A1
:102780000C944217EF92FF920F931F93CF93DF9316
:1027900000D000D000D0CDB7DEB786E0E0E3F2E0B5
:1027A000DE01119601900D928A95E1F7E0903202D8
:1027B000F0903302009134021091350210923202EF
:1027C000109233021092340210923502E11003C0CD
:1027D000FF2009F45DC080912B0290912C020E9491
:1027E0007D18AC0190912E02992339F020910A01B5
:1027F00030E02417350758F04BC020910B018AE0D8
:10280000289F900111242417350718F041C09F3FDD
:1028100019F09F5F90932E02EE2061F00E945A12F1
:102820001E1414F09FEF01C091E0989F902D112489
:1028300090933202FF2061F00E945A121F1414F08C
:102840009FEF01C091E0989F902D11249093330247
:10285000309132023323E1F0209133022223C1F080
:1028600045EB3403C0011124992319F090933202EF
:1028700003C081E08093320235EB2303C0011124B1
:10288000992319F09093330203C081E080933302BF
:10289000011103C0112309F45DC0809129029091B8
:1028A0002A020E947D18AC0190912D02992339F0E3
:1028B0002091060130E02417350758F04BC02091D5
:1028C00007018AE0289F900111242417350718F08A
:1028D00041C09F3F19F09F5F90932D02002361F04C
:1028E0000E949912101614F09FEF01C091E0989F7A
:1028F000902D112490933402112361F00E949912BB
:10290000111614F09FEF01C091E0989F902D1124B3
:1029100090933502309134023323E1F02091350257
:102920002223C1F045EB3403C0011124992319F08F
:102930009093340203C081E08093340235EB23038B
:10294000C0011124992319F09093350203C081E04E
:10295000809335028091320281110BC08091330245
:10296000811107C080913402811103C0809135022A
:1029700081110E94A413EB82FC820D831E8386E0EA
:10298000FE013196A0E3B2E001900D928A95E1F745
:1029900026960FB6F894DEBF0FBECDBFDF91CF9164
:1029A0001F910F91FF90EF900895E0E3F2E086E031
:1029B000DF011D928A95E9F710922E0210922D02E6
:1029C00010922F020895CF93DF93EC01FB018281D7
:1029D000882309F43CC1C430FDE5DF0760F4CB3F38
:1029E0009CE5D90788F49E0122503C4524313105ED
:1029F00008F02EC109C0C236EDE5DE0729F0C63A5F
:102A0000FDE5DF0709F024C10E94240D90935002D8
:102A100080934F02C1318CE5D80709F4C6C008F095
:102A200042C0C930ECE5DE0709F49BC000F5C530B3
:102A30008CE5D80709F485C078F4C330ECE5DE07EF
:102A400009F478C008F07AC0C230DC4509F0F5C05E
:102A500080914F028160EFC0C7309CE5D90709F42F
:102A600078C008F07AC080914F028061E4C0CD3018
:102A7000FCE5DF0709F487C058F4CB309CE5D907A3
:102A800009F479C008F07BC080914F0288606FC064
:102A9000CF30FCE5DF0709F480C008F082C08091E8
:102AA0004F02877FC8C0CE3F9CE5D90709F471C0AB
:102AB00000F5C531FCE5DF0709F485C068F4C331D2
:102AC0009CE5D90709F475C008F095C00E94D506A9
:102AD00080914F028F77AFC0CC3FFCE5DF07A9F1B3
:102AE00008F054C0CB3FDC4509F0A7C080915002EC
:102AF00040C0C230EDE5DE0709F489C058F4C115C5
:102B00008DE5D80709F45AC008F069C080915002D9
:102B100082602FC0C236EDE5DE0709F47CC0C63AFC
:102B2000FDE5DF0709F481C0C330DD4509F085C04C
:102B300080E06EC080914F0282607DC080914F0224
:102B400016C080914F02886076C0809150028260EA
:102B50004FC080914F0280626EC080914F028064AE
:102B60006AC00E94D50680914F02806864C084606C
:102B700062C081603DC080914F028E7F5CC08091B9
:102B80004F028D7F58C080914F0216C08091500235
:102B900018C0809150028D7F2BC080914F028F7E94
:102BA0004AC080914F028F7D46C080914F028F7B3B
:102BB00042C080914F02877F8B7F3DC08091500241
:102BC0008D7F8E7F15C080914F0282FB222720F9D6
:102BD00091E0922790FB82F990FB83F92CC08091C1
:102BE0005002982F909591708E7F892B90FB81F9E0
:102BF0008093500222C00E94D50680914F0287FB2D
:102C0000222720F991E0922790FB87F914C081E0F8
:102C10000E94BB0D12C080914F0284FB222720F935
:102C200091E0922790FB84F906C080914F02982F83
:102C3000909590FB80F980934F0280914F02909184
:102C400050020E94350D0E94D50680E001C081E04F
:102C5000DF91CF910895CF93DF9386319C4541F565
:102C6000EB010E94280C982F8A812091020130915B
:102C70000301882379F09A7A81E009F480E0809357
:102C80003602911102C069E201C065E3C9010E94E8
:102C9000BE170AC080913602811102C069E201C0EC
:102CA00065E3C9010E94C0170E946A0C80E001C060
:102CB00081E0DF91CF9108950F931F93CF93DF931E
:102CC000C42FD22FFC0182818823C9F0409339029E
:102CD0000E946518909338028093370280E28C0F2F
:102CE000883008F057C0C77081E001C0880FCA95CE
:102CF000EAF7DF91CF911F910F910C9432048091EC
:102D00003902481330C080913702909138020E94F6
:102D10007D18883C910538F510E21D0FCD17B9F0EC
:102D200080E28C0F883040F4C77081E001C0880FCA
:102D3000CA95EAF70E943904183028F581E09D2FE2
:102D4000977001C0880F9A95EAF70E943204802F8D
:102D50000E9429041830F0F4D77081E001C0880F78
:102D6000DA95EAF70AC080E28C0F883098F4C770D1
:102D700081E001C0880FCA95EAF7DF91CF911F91DA
:102D80000F910C943904802FDF91CF911F910F91F7
:102D90000C942904DF91CF911F910F9108950F9307
:102DA0009C01CB01243F4CE5340731F188F4293DE7
:102DB000FCE53F07D9F02A3D4CE5340779F1283D81
:102DC0003C45A9F506E221EE41EE68ED7CE52BC01D
:102DD000263FFCE53F07E1F0A8F0273F3C4539F5E9
:102DE00007E225EE46EE67EF7CE51DC007E225EE23
:102DF00045EE69ED7CE517C006E221EE40EE64EF9A
:102E00007CE511C007E225EE44EE65EF7CE50BC0E2
:102E100006E221EE42EE66EF7CE505C008E221E025
:102E200045EE6AED7CE50E945C1680E008C0FC017E
:102E30008281882319F01092390201C081E00F913C
:102E4000089590938F0180938E01089590933F028F
:102E500080933E020895E0913E02F0913F02309748
:102E600021F00190F081E02D099480E00895E09137
:102E70003E02F0913F02309721F00280F381E02D75
:102E800009940895E0913E02F0913F02309739F0A5
:102E900022E0DC012C930480F581E02D0994089553
:102EA00020913C0230913D022817390771F0909330
:102EB0003D0280933C02E0913E02F0913F02309748
:102EC00021F00680F781E02D0994089520913A02BF
:102ED00030913B022817390771F090933B028093A1
:102EE0003A02E0913E02F0913F02309721F00084D7
:102EF000F185E02D09940895FC01329697E080E079
:102F0000915029F021912223D9F38F5FF9CF0895B1
:102F1000662349F0FC01329608962191621729F048
:102F2000E817F907D1F780E0089581E008959C0142
:102F3000FC0132969FEF80E04191461789F09F3F58
:102F400019F4411101C0982F8F5F8630A9F79F3F78
:102F500039F0F901E90FF11D97FDFA9562830895A3
:102F600008959C012A5F3F4FFC014281461301C036
:102F70001282019682179307B9F708950C94971758
:102F80000C94B117029626E0FC0111922A95E9F7FC
:102F9000089508950C94C91783E0809340020C941F
:102FA000CA17811102C081E001C082E08093400213
:102FB0000C94CA170C94D11781E0809340020C94B2
:102FC000CA170C94DC1708950C94E3170C94E417BB
:102FD0000C94E3170C94E3170C94E317CF930E941F
:102FE000EA170E94BB110E94E817C0E08C2F0E94D4
:102FF000E510892B29F4CF5FC530C1F780E001C00F
:1030000081E0CF91089508951F920F920FB60F920D
:1030100011248F939F93AF93BF93809141028111AD
:1030200013C08091650290916602A0916702B091F1
:1030300068024196A11DB11D8093650290936602BE
:10304000A0936702B0936802BF91AF919F918F9157
:103050000F900FBE0F901F90189580916D028430D5
:1030600031F10E9485021092410220E488E190E053
:103070000FB6F894A895809360000FBE209360006F
:1030800083B7817F846083BF83B7816083BF789477
:10309000889583B78E7F83BF0FB6F894A8958091EB
:1030A0006000886180936000109260000FBE0895F8
:1030B0000E94D5060C94890282E084BD93E095BD00
:1030C0009AEF97BD80936E0008952FB7F894809182
:1030D000650290916602A0916702B09168022FBFCD
:1030E00008952FB7F89460916502709166028091FF
:1030F0006702909168022FBF08959C014FB7F89422
:103100008091650290916602A0916702B091680279
:103110004FBF821B930B089578941F920F920FB6A6
:103120000F9211248F939F93AF93BF938091650269
:1031300090916602A0916702B09168020196A11D6C
:10314000B11D8093650290936602A0936702B093CD
:103150006802BF91AF919F918F910F900FBE0F901A
:103160001F90189581E08093E00080E28093D80062
:103170001092C9008FE19EE40197F1F700C00000B2
:1031800087E090EBDC018093760290937702A09326
:103190007802B09379029CE088E10FB6F894A89584
:1031A000809360000FBE90936000FFCF80914D022E
:1031B0000895089522E02093E9002FEF3091E80070
:1031C000215035FD06C035ED3A95F1F7000021118B
:1031D000F5CF2091E80025FF0BC040E050E066E00D
:1031E00070E00E94041B8091E8008E778093E800D5
:1031F0000895CF93DF9321E02093E9002FEF3091E2
:10320000E800215035FD06C035ED3A95F1F7000094
:103210002111F5CF2091E80025FF14C0EC0140E01A
:1032200050E068E070E00E94041B8091E8008E7717
:103230008093E80088E0FE01A5E4B2E001900D92E1
:103240008A95E1F7DF91CF910895809342027093C0
:1032500044026093430280916D02843001F582E064
:103260008093E9008FEF9091E800815095FD06C0B2
:1032700095ED9A95F1F700008111F5CF8091E80066
:1032800085FF0DC040E050E063E070E082E492E032
:103290000E94041B8091E8008E778093E8000895D7
:1032A000BC0184E00C942519BC0183E00C94251921
:1032B00080916C02811109C00E94951C0E94F21C31
:1032C0008091E20084608093E200089510926C0285
:1032D00008950C94E1176091690281E0611101C0C9
:1032E00080E00C94CC1790916D0281E0943009F04D
:1032F00080E0609169020C94D11742E061EC81E0BA
:103300000E940E1C42E261EC82E00E940E1C909131
:103310006D0281E0943009F080E0609169020C94C4
:10332000DA1780916F02833009F461C030F4813084
:1033300071F0823009F49AC008958A3009F486C089
:103340008B3009F46CC0893009F0A8C020C080918E
:103350006E02813A09F0A2C08091E800877F8093D5
:10336000E8008091720290917302892B21F468E049
:1033700085E492E003C060E080E090E070E00E94AD
:103380004F1B8091E8008B778093E800089580912F
:103390006E02813209F082C08091720290917302B4
:1033A000029708F07BC08091E800877F8093E80057
:1033B0008091E80082FD05C080916D028111F8CFF7
:1033C0006DC02091F3008091F20090E0922B029763
:1033D00031F48091F100813011F0863021F4809138
:1033E000F10080934D028091E8008B7753C080916B
:1033F0006E02813A09F052C080917202909173027C
:10340000892B09F04BC08091E800877F8093E8000A
:103410008091E80080FFFCCF8091180136C0809138
:103420006E028132D9F58091720290917302892BDC
:10343000A9F58091E800877F8093E8000E94431CF3
:1034400080917002809318010C94D50680916E02D1
:10345000813221F58091E800877F8093E8000E9407
:10346000431C8091710280934E02089580916E02F8
:10347000813AA1F48091E800877F8093E8008091F1
:10348000E80080FFFCCF80914E028093F100809194
:10349000E8008E778093E8000C94431C089584B76D
:1034A000877F84BF0FB6F894A895809160008861EB
:1034B00080936000109260000FBE90E080E80FB62D
:1034C000F89480936100909361000FBE0C94DC1718
:1034D0000E94951C0E94F21CE2EEF0E08081846064
:1034E000808378940C94871F8CE091E00C942617CD
:1034F00080916D028530A9F480916D02853079F458
:103500000E942D1880916B028823B1F30E94EE1760
:10351000882391F30E94EE1A0E94D506EDCF0C94F9
:103520005818089508950C94951A292F332723309D
:103530003105C9F060F42130310581F022303105C8
:1035400009F044C08BE390E02EE132E043C0213229
:103550003105E1F02232310549F138C082E190E0D5
:1035600029E532E037C099278130910549F028F0EC
:10357000029761F5E0EFF1E005C0EAE1F2E002C098
:10358000E4E0F2E0849190E09F0124C061157105B0
:1035900041F061307105D1F489E090E029E432E036
:1035A00019C089E090E020E332E014C06115710594
:1035B00041F06130710551F48BE790E02BE632E089
:1035C00009C080E490E026EE32E004C080E090E0A4
:1035D00020E030E0FA0131832083089580E189BD45
:1035E00082E189BD09B400FEFDCF8091D8008F7DB6
:1035F0008093D8008091E00082608093E000809109
:10360000E00081FDFCCF0895CF92DF92EF92FF9210
:103610000F931F93CF93DF93EC018B017A010E94EC
:10362000621C811133C0E114F10439F0F70180818B
:103630009181081B190BC80FD91FC12CD12C011562
:10364000110519F18091E80085FD16C08091E80010
:103650008E778093E800E114F10449F0F70180814E
:103660009181C80ED91ED182C08285E00FC00E9410
:10367000621C882321F30AC089918093F1000150D4
:103680001109FFEFCF1ADF0ADACF80E0DF91CF9187
:103690001F910F91FF90EF90DF90CF9008952091B0
:1036A0007402309175022617370748F061157105CD
:1036B00039F42091E8002E772093E80001C0B90189
:1036C000FC0120E06115710579F180916D0288237C
:1036D000F1F18530F1F18091E80083FD3CC08091EB
:1036E000E80082FD2EC08091E80080FFEBCF2091A2
:1036F000F3008091F20090E0922B6115710551F07A
:103700008830910538F421912093F10061507109BE
:103710000196F3CF21E0089709F020E08091E800BE
:103720008E778093E800CECF2111CFCF0AC0809151
:103730006D02882361F0853061F08091E80083FD9F
:103740000AC08091E80082FFF2CF80E0089582E015
:10375000089583E0089581E00895209174023091E6
:1037600075022617370748F06115710539F4209165
:10377000E8002E772093E80001C0B901FC0120E0A9
:103780006115710591F180916D02882309F440C0A3
:10379000853009F43FC08091E80083FD3DC08091F1
:1037A000E80082FD2FC08091E80080FFE9CF2091E2
:1037B000F3008091F20090E0922B6115710559F0B1
:1037C0008830910540F424912093F10031966150A6
:1037D00071090196F2CF21E0089709F020E080916D
:1037E000E8008E778093E800CBCF2111CCCF0AC0C0
:1037F00080916D02882361F0853061F08091E8004E
:1038000083FD0AC08091E80082FFF2CF80E0089536
:1038100082E0089583E0089581E00895982F97301D
:1038200068F59093E900981739F07091EC002091B9
:10383000ED005091F00003C0242F762F50E021FDC1
:1038400002C09F5FECCF3091EB003E7F3093EB00E6
:103850003091ED003D7F3093ED003091EB00316011
:103860003093EB007093EC002093ED005093F00048
:103870002091EE0027FDE5CF80E008958F708093C2
:10388000E90081E0089580916E0287FF11C0809168
:10389000E80082FD05C080916D028111F8CF11C052
:1038A0008091E8008B770BC080916D02882349F0EE
:1038B0008091E80080FFF8CF8091E8008E778093B8
:1038C000E80008952091E4003091E50095E64091EC
:1038D000EC00842F817040FF23C08091E80080FDC0
:1038E0001DC080916D02882399F0853099F08091F8
:1038F000EB0085FD11C04091E4005091E5002417D4
:10390000350729F3915011F09A01E1CF84E0089531
:1039100082E0089583E0089581E0089580E00895AD
:103920004091E80042FFDDCF08950E94031D0E94F0
:103930000B1DE0EEF0E0808181608083E8EDF0E037
:1039400080818F77808319BCA7EDB0E08C918E7F4A
:103950008C9380818F7E808310926C0208950F93E8
:103960001F93CF93DF930E94031D0E940B1DC8ED90
:10397000D0E088818F778883888180688883888178
:103980008F7D888319BC10926D021092690210928B
:103990006B0210926A0200EE10E0F80180818B7FCA
:1039A000808388818160888342E060E080E00E94BB
:1039B0000E1CE1EEF0E080818E7F8083E2EEF0E08D
:1039C000808181608083808188608083F80180812C
:1039D0008E7F8083888180618883DF91CF911F9162
:1039E0000F910895E8EDF0E080818F7E8083E7ED10
:1039F000F0E080818160808384E082BF81E08093F9
:103A00006C020C94AF1CE8EDF0E080818E7F808327
:103A10001092E20008951092DA001092E1000895E9
:103A20001F920F920FB60F9211242F933F934F9333
:103A30005F936F937F938F939F93AF93BF93EF9316
:103A4000FF938091E10082FF0BC08091E20082FF32
:103A500007C08091E1008B7F8093E1000E94861F68
:103A60008091DA0080FF1FC08091D80080FF1BC0CA
:103A70008091DA008E7F8093DA008091D90080FFF8
:103A80000DC080E189BD82E189BD09B400FEFDCF92
:103A900081E080936D020E94581905C019BC1092F4
:103AA0006D020E9466198091E10080FF19C080912B
:103AB000E20080FF15C08091E2008E7F8093E200DB
:103AC0008091E20080618093E2008091D800806262
:103AD0008093D80019BC85E080936D020E946B1919
:103AE0008091E10084FF30C08091E20084FF2CC00F
:103AF00080E189BD82E189BD09B400FEFDCF8091DE
:103B0000D8008F7D8093D8008091E1008F7E8093D4
:103B1000E1008091E2008F7E8093E2008091E200DC
:103B200081608093E20080916902882311F084E033
:103B300007C08091E30087FD02C081E001C083E0FF
:103B400080936D020E9473198091E10083FF29C068
:103B50008091E20083FF25C08091E100877F809300
:103B6000E10082E080936D02109269028091E10091
:103B70008E7F8093E1008091E2008E7F8093E2004F
:103B80008091E20080618093E20042E060E080E0AA
:103B90000E940E1C8091F00088608093F0000E94CB
:103BA0006919FF91EF91BF91AF919F918F917F9193
:103BB0006F915F914F913F912F910F900FBE0F909A
:103BC0001F9018951F920F920FB60F9211242F93EA
:103BD0003F934F935F936F937F938F939F93AF9395
:103BE000BF93CF93DF93EF93FF93C091E900CF7022
:103BF0008091EC00D82FD17080FDD0E81092E900C0
:103C00008091F000877F8093F00078940E94261EB8
:103C10001092E9008091F00088608093F000CD2B35
:103C2000CF70C093E900FF91EF91DF91CF91BF91E9
:103C3000AF919F918F917F916F915F914F913F9144
:103C40002F910F900FBE0F901F9018951F93CF9339
:103C5000DF93CDB7DEB7AA970FB6F894DEBF0FBEDD
:103C6000CDBFEEE6F2E08091F100819322E0E637ED
:103C7000F207C9F70E9491198091E80083FF2EC1D5
:103C800080916E0290916F02492F50E04A305105A9
:103C900008F024C1FA01EE59FF4F0C94B61F80388A
:103CA00021F0823809F01AC108C080916A0290910F
:103CB0006B02992389F082600FC0809172028F702D
:103CC000873008F00BC18093E9008091EB0085FB01
:103CD000882780F91092E9009091E800977F9093EF
:103CE000E8008093F1001092F100D1C0282F2D7FC1
:103CF00009F0F4C0882319F0823061F0EFC08091A0
:103D00007002813009F0EAC0933009F080E08093BE
:103D10006B022EC08091700281112AC080917202C4
:103D20008F702FEF280F263008F0D8C08093E9005D
:103D30002091EB0020FF1CC0933021F48091EB0018
:103D4000806214C09091EB0090619093EB0021E0B1
:103D500030E0A90102C0440F551F8A95E2F7409355
:103D6000EA001092EA008091EB0088608093EB00FB
:103D70001092E9008091E800877F8093E8000E941C
:103D8000431CACC08111AAC0109170021F778091B2
:103D9000E3008078812B8093E3008091E800877FA7
:103DA0008093E8000E94431C8091E80080FFFCCFD4
:103DB0008091E30080688093E300111102C082E0EB
:103DC00001C083E080936D0289C08058823008F082
:103DD00085C080917002909171028C3D53E09507EF
:103DE00079F583E08A838AE289834FB7F894DE010C
:103DF000139620E03EE051E2E32FF0E050935700AD
:103E0000E49120FF03C0E295EF703F5FEF708E2FCB
:103E100090E0EA3010F0C79601C0C0968D939D9354
:103E20002F5F243149F74FBF8091E800877F80934F
:103E3000E8006AE270E0CE0101960E944F1B16C0B6
:103E40006091720270917302AE014F5F5F4F0E94EA
:103E5000931ABC01892B09F441C09091E800977F27
:103E60009093E80089819A810E94AD1B8091E800BF
:103E70008B778093E80032C0803881F58091E8002C
:103E8000877F8093E800809169028093F1008091A0
:103E9000E8008E7772CF811121C0809170029091DD
:103EA000710299270297D4F48091E800877F80936C
:103EB000E80080917002809369020E94431C809107
:103EC0006902811106C08091E30087FD02C081E094
:103ED00001C084E080936D020E947D198091E8000A
:103EE00083FF0AC08091E800877F8093E80080917B
:103EF000EB0080628093EB00AA960FB6F894DEBFC9
:103F00000FBECDBFDF91CF911F9108950895CF933C
:103F100080916D028823A1F0C091E900CF7090914B
:103F2000EC00892F817090FD80E8C82B1092E90089
:103F30008091E80083FD0E94261ECF70C093E900A7
:103F4000CF91089597FB072E16F4009407D077FDC4
:103F500009D00E94BC1F07FC05D03EF490958195C6
:103F60009F4F0895709561957F4F0895EE0FFF1F45
:103F70000590F491E02D0994AA1BBB1B51E107C0E9
:103F8000AA1FBB1FA617B70710F0A61BB70B881FE9
:103F9000991F5A95A9F780959095BC01CD01089578
:103FA000FB01DC0104C08D910190801921F4415086
:103FB0005040C8F7881B990B0895F999FECF92BD20
:103FC00081BDF89A992780B50895A8E1B0E042E054
:103FD00050E00C941120262FF999FECF92BD81BD9F
:103FE000F89A019700B4021639F01FBA20BD0FB637
:103FF000F894FA9AF99A0FBE08950396272F0E9413
:10400000EC1F0E94EB1F252F0E94EC1F242F0C9405
:10401000EC1F0196272F0E94EC1F0C94EB1FDC0174
:10402000CB01FC01F999FECF06C0F2BDE1BDF89AC3
:10403000319600B40D9241505040B8F70895F8946D
:02404000FFCFB0
:10404200C8000902280850011E0A1401D618F918DE
:10405200DA1854195019D91801E200E900EA00B53A
:1040620000B600B700CD008301CC008A0192019412
:10407200012102230224022502260227022A02B378
:1040820000B4006F007000818283E200E900EA0060
:10409200B500B600B700CD008301CC008A019201C1
:1040A20094012102230224022502260227022A0267
:1040B200B300B4006F007000818283F0F1F4F5F672
:0E40C2009496973435366667F79091929395F1
:00000001FF
